:020000040000FA
:1000000083160030850000308600803081009B011F
:10001000831207309F0099205F2099208F29820743
:10002000000006345B344F3466346D347D3407345D
:100030007F346F343F3477347C3439345E347934F0
:1000400071346F34763406341E34383437343F34E8
:100050007334673450346D3478343E346E348034C5
:100060004034083401344834FF34000000000000FC
:100070000000000000000034A00B3C280034000009
:10008000A00B3F2800340430A1000000A00B45283D
:10009000A10B452800340A30A1000000A00B4D2818
:1000A000A10B4D2800340130A400A30B5528A40B4C
:1000B00055280034A30B5A28A40B5A2800340630C4
:1000C000C0005B30C1004030C2005E30C30006306B
:1000D000C4006F30C5000630C6007830C700083055
:1000E000C8005030C9003E30CA003730CB0037302E
:1000F000CC000630CD003730CE006F30CF00083056
:10010000D0006D30D1000630D2006F30D3003730D0
:10011000D4000830D5007C30D6006E30D7000830CF
:10012000D8007830D9007930DA00DA2081215A21DC
:1001300000344F30A0002130840000308000840A59
:10014000A00B9D28003405163520051235200034FB
:100150000830AB0085018503860186036018051011
:10016000611885106218051163188511641806104E
:100170006518861066180611671886116818061229
:10018000691886126A1806136B188613A3203C2080
:10019000E00CE10CE20CE30CE40CE50CE60CE70CE3
:1001A000E80CE90CEA0CEB0CAB0BAA28FF3085003D
:1001B000860000348316203085008312A320851E1C
:1001C000DE28A320003483160513831205173F2071
:1001D0008316051783124B203F20051FF128A50128
:1001E000003425180034A601831605138312051761
:1001F0003F208316051783123F203F20A60A051BC8
:10020000FC28A60B0529A5140034A60B09292515E1
:100210000034A60B0D29A5150034A60B11292516AF
:100220000034A5160034251800342514A80A28081F
:100230000F20DB00FF3A031D0034DB01A801162963
:100240002518003425142808013A031D2A292430D2
:10025000A8002029A80328080F20DB000034251857
:10026000003425140A30A200503084000008003AFF
:1002700003193E29840AA20B3629422928080F2097
:10028000800000344008003A031D00341A30A200F8
:1002900040308400000884038000840A840AA20B92
:1002A0004A295B08D90000342518003425141C3075
:1002B00092000034BF01DB013530F2006030F40001
:1002C0002030F0007208F3007408F5000C30F600DE
:1002D000730884000008F10075088400710880002C
:1002E000F30AF50AF60B6829DA20A820F00B622938
:1002F000F20A7208543A031D6029A508031D5C29FF
:1003000000340C30A0005030840000080412841621
:10031000800004168412840AA00B85290034DA2098
:100320008121A820E320A50803198F29A51C9A295B
:1003300013218F29251D9E2920218F29A51DA22942
:100340002F218F29251EA62954218F29A51A5A2924
:020350008F29F3
:02400E00503F21
:00000001FF
